:10000000AC28FF3FFF3FFF3F0E3003138312FA007F
:10001000FA0B082800000800031383129F01C03068
:100020009F04403083161F04F00070089F0080304A
:1000300070049F0083124908F000F00D7010F00D5D
:100040007010F00D701070089F041F1404201F150D
:1000500000301F190130F2007208013A031D3228E6
:10006000000028281E08F200F3017208F300F201D4
:100070007208CA007308CB0083161E08720483122C
:10008000CA007308CB000030CB041F104A08F000F0
:100090004B08F100080003138312FB01FA01F90178
:1000A0008030F800F10CF00C031C5F287408F9078D
:1000B00075080318750FFA070318FB0A0310F01FE1
:1000C00067287408FA0775080318750FFB07FB0CFF
:1000D000FA0CF90CF80C031C52287B08F3007A0880
:1000E000F2007908F1007808F00008000313831289
:1000F000F801F9011030FC00710DF80DF90D7408CC
:10010000F8027508031C750FF90203188E2874088D
:10011000F80775080318750FF9070310F00DF10DB6
:10012000FC0B7C280800031383127008F100F00117
:100130000830FC007108F40C0318A228FC0B9B2863
:10014000F10100340310A728F40C0318F107F10C97
:10015000F00CFC0BA42808000730031383169C0046
:1001600030308500860110309B008D3083129F0057
:1001700083169F01FF3083128600A001A101A20116
:100180002208323C031CED280D3085000630FA00B1
:10019000FA0BC82800000E3085000630FA00FA0B72
:1001A000CF2800000B3085000630FA00FA0BD62865
:1001B0000000073085000630FA00FA0BDD28000049
:1001C0000F3085000630FA00FA0BE4280000220800
:1001D000323A0319ED28A20AC028A001A101043077
:1001E000C9000C207008A3007108A400D6220313D4
:1001F00083122308F0002408F1006430F400F501B4
:100200004B200630F4007008C5007108C600740861
:100210000319112903138312C60CC50CC613FF3F23
:100220000829031383124508A5004608A6002308E1
:10023000F0002408F1000A30F400F5014B200630EC
:10024000F4007008BD007108BE00740803192F295E
:1002500003138312BE0CBD0CBE13FF3F26290313EC
:1002600083123D08A7003E08A8006430F400F501A1
:100270003D08F0003E08F10076207008A90000302B
:10028000F1006430F400F5014B207008C3007108E0
:10029000C4004308AD004408AE004308BD02031C7F
:1002A000BE034408BE020A30F400F5013D08F00028
:1002B0003E08F10076207008AA000030F1000A30F4
:1002C000F400F5014B207008C1007108C20041081C
:1002D000AF004208B00041083D02F0004208031C94
:1002E000013F3E02F1007008AB000A30F400932099
:1002F0007008BF003F08B1004308F0004408F10057
:100300000A30F400F5014B2070084502BD00710869
:10031000031C013F4602BE004108F0004208F10004
:100320000A30F400F5014B2070083D02F00071081E
:10033000031C013F3E02F1003F08F002031CF103E1
:100340007008AC0003138312A20103138312220866
:10035000033C031C6C2A2930F0002208F0077008C7
:1003600084000008F200031383127208003A031D90
:10037000BF29DD3003138312B200B3012B2A03130C
:1003800083127208013A031DCB291830031383121C
:10039000B200B3012B2A031383127208023A031D21
:1003A000D729753003138312B200B3012B2A03132C
:1003B00083127208033A031DE32979300313831271
:1003C000B200B3012B2A031383127208043A031DEF
:1003D000EF29B83003138312B200B3012B2A0313A1
:1003E00083127208053A031DFB29E93003138312B7
:1003F000B200B3012B2A031383127208063A031DBD
:10040000072AF93003138312B200B3012B2A031316
:1004100083127208073A031D132AD830031383127C
:10042000B200B3012B2A031383127208083A031D8A
:100430001F2AFD3003138312B200B3012B2A0313CA
:1004400083127208093A031D2B2AED30031383121D
:10045000B200B3012B2A031383122208003A031DB2
:10046000382A031383123208B4003308B500622A15
:10047000031383122208013A031D452A0313831232
:100480003208B6003308B700622A03138312220829
:10049000023A031D552A0230031383123207B800B3
:1004A00033080318013FB900622A0313831222089C
:1004B000033A031D622A031383123208BA00330879
:1004C000BB00622A031383122208033A03196C2A21
:1004D00003138312A20AA52903138312BC01031379
:1004E00083123C08643C031CD12A340886000D307A
:1004F00085000630FA00FA0B7B2A00000F308500D9
:100500000130FA00FA0B822A00000000360886004B
:1005100020080E3FF00000300318013F2107F100D2
:10052000700885000630FA00FA0B942A00000F309C
:1005300085000130FA00FA0B9B2A00000000380801
:1005400086000B3085000630FA00FA0BA52A000061
:100550000F3085000130FA00FA0BAC2A00000000D1
:100560003A0886002008073FF00000300318013FDA
:100570002107F100700885000630FA00FA0BBE2A48
:1005800000000F3085000130FA00FA0BC52A000088
:1005900000003C08643A0319D12A03138312BC0AF1
:1005A0006F2A0F30031383128500ED2802300313E6
:1005B00083122402031DDE2AA03023020318E62A38
:1005C000403003138312A000A1010800031383121B
:1005D0002408033C031DEE2A2308C03C0318F62A16
:1005E000803003138312A000A1010800F728F72A26
:04400E00583FFFFF19
:00000001FF
